:0200000480007A
:100000006F008004732F2034930F80006308FF0378
:10001000930F90006304FF03930FB0006300FF038E
:10002000130F000063040F0067000F00732F2034CC
:1000300063540F006F00400093E19153171F0000BD
:1000400023223FFC6FF09FFF93000000130100008C
:10005000930100001302000093020000130300004C
:100060009303000013040000930400001305000034
:10007000930500001306000093060000130700001C
:100080009307000013080000930800001309000004
:1000900093090000130A0000930A0000130B0000EC
:1000A000930B0000130C0000930C0000130D0000D4
:1000B000930D0000130E0000930E0000130F0000BC
:1000C000930F0000732540F16310050097020000B4
:1000D000938202017390523073500018970200000F
:1000E00093824202739052309B021000939252030B
:1000F0009382F2FF7390023B9302F0017390023AF5
:100100007350403097020000938242017390523046
:10011000735020307350303093010000970200007C
:10012000938282EE73905230130510001315F5017F
:10013000635C05000F00F00F930110009308D005D9
:10014000130500007300000093020000638A0200A0
:1001500073905210B7B200009B82921073902230BD
:100160007350003097020000938242017390123462
:10017000732540F17300203097200000938080E8C1
:10018000370155001B0151051311010113015105E0
:10019000131111011301A10A23B0200003B70000BD
:1001A000B70355009B835305939303019383530532
:1001B000939313019383A30A930120006310776044
:1001C00097200000938000E43701D5FF1B01510503
:1001D00013110101130151051311D1001301B100D5
:1001E0001311C100130101A023B4200003B7800044
:1001F000B703D5FF9B835305939303019383530563
:100200009393D3009383B3009393C300938303A08A
:10021000930130006314775A97200000938080DEAA
:10022000370155001B0151051311D1001301B10015
:100230001311C100130111A01311C100130101AA70
:1002400023B8200003B70001B70355009B83530573
:100250009393D3009383B3009393C300938313A02A
:100260009393C300938303AA9301400063187754C8
:1002700097200000938000D93701FDFF1B01510535
:10028000131101011301510513110101130151054E
:100290001311D1001301A10023BC200003B780017A
:1002A000B703FDFF9B83530593930301938353058A
:1002B00093930301938353059393D3009383A300F4
:1002C00093015000631C774E97200000938000D765
:1002D000370155001B01510513110101130151058F
:1002E000131111011301A10A23B420FE03B780FEEC
:1002F000B70355009B8353059393030193835305E1
:10030000939313019383A30A930160006318774AC0
:1003100097200000938080D23701D5FF1B01510543
:1003200013110101130151051311D1001301B10083
:100330001311C100130101A023B820FE03B700FF71
:10034000B703D5FF9B835305939303019383530511
:100350009393D3009383B3009393C300938303A039
:1003600093017000631C774497200000938000CDB8
:10037000370155001B0151051311D1001301B100C4
:100380001311C100130111A01311C100130101AA1F
:1003900023BC20FE03B780FFB70355009B835305A2
:1003A0009393D3009383B3009393C300938313A0D9
:1003B0009393C300938303AA930180006310774053
:1003C00097200000938080C73701FDFF1B01510576
:1003D00013110101130151051311010113015105FD
:1003E0001311D1001301A10023B0200003B70000B6
:1003F000B703FDFF9B835305939303019383530539
:1004000093930301938353059393D3009383A300A2
:10041000930190006314773A97200000938080C284
:10042000377124001B01D18A1311E100130191C01F
:100430001311D100130151341311C100130181674D
:10044000138200FE2330220283B20000B77324001F
:100450009B83D38A9393E300938393C09393D300B6
:10046000938353349393C300938383679301A000D2
:1004700063967234972000009380C0BC3741B0006F
:100480001B0111261311C1001301B1301311F1002A
:10049000130131211311C100130181099380D0FF91
:1004A000A3B5200017220000130242BA83320200D3
:1004B000B743B0009B8313269393C3009383B33059
:1004C0009393F300938333219393C300938383091E
:1004D0009301B0006394722E9301C00013020000D8
:1004E000B7D0BB0A9B80D0CD17210000130181B18A
:1004F0002330110003370100B7D3BB0A9B83D3CD50
:10050000631E772A1302120093022000E31A52FCA2
:100510009301D00013020000B7C0AB0A9B80D0CC7F
:1005200017210000130101AE130000002334110055
:1005300003378100B7C3AB0A9B83D3CC6310772802
:100540001302120093022000E31852FC9301E00012
:1005500013020000B7C0AA0D9B80C0BC1721000089
:10056000130141AA130000001300000023381100FA
:1005700003370101B7C3AA0D9B83C3BC6310772463
:100580001302120093022000E31652FC9301F000C4
:1005900013020000B7B0DA0D9B80C0BB130000004F
:1005A00017210000130101A6233C1100033781012C
:1005B000B7B3DA0D9B83C3BB63127720130212001B
:1005C00093022000E31852FC930100011302000083
:1005D000B7B0DD0C9B80B0AB13000000172100000A
:1005E000130141A21300000023301102033701025E
:1005F000B7B3DD0C9B83B3AB6312771C13021200FD
:1006000093022000E31652FC930110011302000034
:10061000B7E0CD0C9B80B0AA1300000013000000CF
:10062000172100001301019E2334110203378102B8
:10063000B7E3CD0C9B83B3AA6312771813021200A1
:1006400093022000E31652FC9301200113020000E4
:10065000172100001301019BB72011009B8030235C
:100660002330110003370100B72311009B8333238C
:10067000631677141302120093022000E31A52FC4F
:10068000930130011302000017210000130181972C
:10069000B71001309B80302213000000233411007A
:1006A00003378100B71301309B833322631877101F
:1006B0001302120093022000E31852FC9301400140
:1006C00013020000172100001301C193B71000337B
:1006D0009B8020121300000013000000233811003B
:1006E00003370101B71300339B8323126318770C80
:1006F0001302120093022000E31652FC93015001F2
:1007000013020000172100001301C18F1300000025
:10071000B70030239B802011233C11000337810157
:10072000B70330239B832311631A77081302120047
:1007300093022000E31852FC9301600113020000B1
:10074000172100001301018C13000000B7003322B1
:100750009B801001130000002330110203370102B7
:10076000B70333229B831301631A77041302120029
:1007700093022000E31652FC930170011302000063
:10078000172100001301018813000000130000006E
:10079000B73023129B8010002334110203378102EB
:1007A000B73323129B831300631A770013021200DE
:1007B00093022000E31652FC631030020F00F00F8A
:1007C000638001009391110093E111009308D0051B
:1007D00013850100730000000F00F00F930110005B
:1007E0009308D0051305000073000000731000C0CB
:0C07F000000000000000000000000000FD
:1010000000000000000000000000000000000000E0
:1010100000000000000000000000000000000000D0
:1010200000000000000000000000000000000000C0
:1010300000000000000000000000000000000000B0
:081040000000000000000000A8
:10200000EFBEADDEEFBEADDEEFBEADDEEFBEADDEF0
:10201000EFBEADDEEFBEADDEEFBEADDEEFBEADDEE0
:10202000EFBEADDEEFBEADDEEFBEADDEEFBEADDED0
:10203000EFBEADDEEFBEADDEEFBEADDEEFBEADDEC0
:10204000EFBEADDEEFBEADDEEFBEADDEEFBEADDEB0
:040000058000000077
:00000001FF
